:1000000009308A004A290000FF00030E8301A10085
:100010007F08A0000A08A7008A01A00E0408A20019
:100020007708A3007808A4007908A5007A08A6003C
:10003000831383120B1E1E288B1835288C308400E6
:10004000001C24280C183728220884002308F700F5
:100050002408F8002508F9002608FA0027088A0075
:10006000210E8300FF0E7F0E09008A1181288A115C
:1000700052290A108A100A1182070A3478346D3422
:10008000693474342034253475342C342534753473
:100090002034733474346134743465343D3425341D
:1000A000753400340A108A100A118207C034E7340C
:1000B0008C348634A33492349034C73480348334FF
:1000C0008134B034D834A43498349934FF340A10CD
:1000D0008A100A11820720347434723469347334FC
:1000E00061343D34203400340A108A100A1182072A
:1000F0002034743472346934733462343D342034BF
:1001000000348316400F852886284E29000083126C
:10011000AB000308AA009E2031082E18FF3083167A
:10012000C000972880014002031942109728000060
:1001300083122A088300AB0E2B0E46292E148B1334
:100140006400831685308316810083120130831288
:10015000AC0064008101061CAB280108AF008316C7
:10016000480883122F02031C2D2983164908831285
:100170002F0703182D290230AC000730B0006400AF
:1001800081010618C1280108AF00831643088312B5
:100190002F02031C2D298316440883122F070318EE
:1001A0002D2981016400061CD3280108AF008316A5
:1001B000430883122F02031C2D298316450883123E
:1001C0002F0703182D298316440883122F070318BD
:1001D000EC280310B10CEE280314B10CB00BC028AE
:1001E0000310B10C0330AC000530B00081010618DB
:1001F000F7280108AF008316430883122F02031C5F
:100200002D298316440883122F0703182D298101F5
:100210006400061C09290108AF00831643088312F5
:100220002F02031C2D298316450883122F0703185C
:100230002D298316440883122F070318222903103F
:10024000B20C24290314B20CB00BF6280310B20C24
:100250000310B20C0310B20CAE010B118316053063
:100260008316810083128312080000000130831678
:10027000BF00C730E5000130E600E50B4029E60B82
:100280003D29BF0B392900008312080000008316A6
:10029000400F4B294E2983122915831683128B1088
:1002A0008A1124283D08053C031D7529861606126F
:1002B00083162608E500650883125220F80083168D
:1002C000B5006508123C031C7329350883128500AC
:1002D0008316B51E6F298312861771298316831220
:1002E000861375298316B8018312BD08031D97294B
:1002F0008612061683162708E50065088312522029
:10030000F8008316B5006508123C031C95293508D2
:10031000831285008316B51E9129831286179329AF
:1003200083168312861397298316B8018312BD0A98
:100330003D080A3C0319BD01F6308F003C308E00A9
:100340000C108A11242883169B019C131C141A0874
:10035000AD00AD080319B0292D08083C0318C829C1
:100360000330AD009B012D089A009C131C158312CD
:100370000B08F7008B13831655309D00AA309D00A3
:100380009C149C18C1291C11770883128B048316B6
:1003900001309B009C131C141A08AE00AE08031910
:1003A000D5292E08083C0318EE290230AE00013092
:1003B0009B002E089A009C131C1583120B08F70053
:1003C0008B13831655309D00AA309D009C149C18F9
:1003D000E7291C11770883128B04831602309B00D7
:1003E0009C131C141A08AC00AC080319FB292C0838
:1003F0000A3C0318142A0130AC0002309B002C0880
:100400009A009C131C1583120B08F7008B1383169C
:1004100055309D00AA309D009C149C180D2A1C117B
:10042000770883128B04831603309B009C131C14E3
:100430001A08AA002A08093C0318372A0430AA001F
:1004400003309B002A089A009C131C1583120B088A
:10045000F7008B13831655309D00AA309D009C1425
:100460009C18302A1C11770883128B048316831280
:100470008A157E290800DD308400831300080319E3
:100480004F2A0130F800F701F70B442AF80B432AF2
:100490004A30F700F70B4A2A4D2A800B412A080000
:1004A000861606120A308316DD0083123B220800EE
:1004B0000B128B1083160C1083128615FF308500EB
:1004C00083164D0BBB2A8312502283162D08E5009C
:1004D000650883125220F8008316B5006508123CA7
:1004E000031C802A3508831285008316B51E7C2ADA
:1004F000831286177E2A831683128613822A831616
:10050000B80183120A308316CE008230DD008312D8
:100510003B228316CE0B852A8312061686120A30DA
:100520008316DD0083123B2283162E08E500650842
:1005300083125220F8008316B5006508123C031C94
:10054000AF2A3508831285008316B51EAB2A8312A5
:100550008617AD2A831683128613B12A8316B80133
:1005600083120A308316CE008230DD0083123B22D4
:100570008316CE0BB42A83120C10BD01F6308F0007
:100580003C308E0083160C14C03083128B0483160B
:100590004D0BD72A2C08A7001030A6000A30CE0039
:1005A0008230DD0083123B228316CE0BD02A29082D
:1005B0000F39B5003508A7002908F039B500B50E88
:1005C0003508A6000C14F63083128F003C308E00E4
:1005D00083164D0BF52A0A30CE008230DD008312DF
:1005E0003B228316CE0BED2AFE2A0330CE00C83004
:1005F000DD0083123B228316CE0BF72AFF308312D5
:1006000085000616861683160C1083128B10C030D8
:100610008B040800FF308316C00083128B108316F2
:10062000B5018312061C172B8316B50A83122911F4
:1006300008008A15EB2986130830F8001F2B0000EC
:10064000F817322BF8138316E20C8312031886175F
:10065000031C86137817322B7813F80B232B302BBF
:10066000000086171C308400840B342B372BF81BBA
:10067000222B781B2C2B08000A308316E2008312F1
:100680001B238316CE014E08831267208316CE0AE1
:10069000F7007708E20083121B23083083164E020E
:1006A000031D432B0508CE00CF014F08073C031C58
:1006B000732BCE1F612B3130E20083121B23652B7D
:1006C00083163030E20083121B2383164F08033C4D
:1006D000031D6F2B2D30E20083121B2383160310A2
:1006E000CE0DCF0A552BCE014E08831274208316EF
:1006F000CE0AF7007708E20083121B230830831626
:100700004E02031D742B0608CE00CF014F08073C94
:10071000031CA42BCE1F922B3130E20083121B232B
:10072000962B83163030E20083121B2383164F086A
:10073000033C031DA02B2D30E20083121B238316E4
:100740000310CE0DCF0A862B831208008316E0011A
:100750006008831239208316E00AF7007708E20068
:1007600083121B23063083166002031DA82B5D082D
:10077000E0001B30E10078086008E2006430E3002C
:100780006308F80162020318C82B6208F700D42B33
:10079000F7010830E400E20DF70D63087702031853
:1007A000F700F80DE40BCB2B7708E0007808303029
:1007B000031DE12BE11CEA2BE119EA2B611A203021
:1007C000E42BE11161126114F8077808E20083124A
:1007D0001B2383166008E2000A30E3006308F80177
:1007E00062020318F62B6208F700022CF7010830AA
:1007F000E400E20DF70D630877020318F700F80D27
:10080000E40BF92B7708E00078083030031D0E2C3C
:10081000E119142C611C142C611A2030F807780897
:10082000E20083121B2383163030E0076008E200E9
:1008300083121B232C308316E20083121B238316A2
:100840005E08E0001B30E10078086008E2006430D8
:10085000E3006308F80162020318312C6208F70014
:100860003D2CF7010830E400E20DF70D6308770234
:100870000318F700F80DE40B342C7708E000780833
:100880003030031D4A2CE11C532CE119532C611A02
:1008900020304D2CE11161126114F8077808E20054
:1008A00083121B2383166008E2000A30E30063080A
:1008B000F801620203185F2C6208F7006B2CF70145
:1008C0000830E400E20DF70D630877020318F70023
:1008D000F80DE40B622C7708E00078083030031D37
:1008E000772CE1197D2C611C7D2C611A2030F807D2
:1008F0007808E20083121B2383163030E00760087B
:10090000E20083121B230B308316E0006008831281
:1009100039208316E00AF7007708E20083121B23D0
:10092000123083166002031D862C5F08E0001B3026
:10093000E10078086008E2006430E3006308F80131
:1009400062020318A62C6208F700B22CF7010830E7
:10095000E400E20DF70D630877020318F700F80DC5
:10096000E40BA92C7708E00078083030031DBF2C79
:10097000E11CC82CE119C82C611A2030C22CE111ED
:1009800061126114F8077808E20083121B238316B2
:100990006008E2000A30E3006308F801620203180D
:1009A000D42C6208F700E02CF7010830E400E20DD7
:1009B000F70D630877020318F700F80DE40BD72C46
:1009C0007708E00078083030031DEC2CE119F22C98
:1009D000611CF22C611A2030F8077808E2008312BB
:1009E0001B2383163030E0076008E20083121B23CC
:1009F0000B138B138B1BF92C83165F0B3A2D5D08A1
:100A0000003A831203190B2D013A03191A2D033AE8
:100A10000319292D382D0130F70083165E08F800E0
:100A20000319162D0310F70DF80B122D77088312FA
:100A30008504382D0130F70083165E08F80003198D
:100A4000252D0310F70DF80B212D7708831286044E
:100A5000382D0130F70083165E08F8000319342D95
:100A60000310F70DF80B302D770883128704382D0B
:100A7000762D83165D08003A83120319462D013A3C
:100A80000319562D033A0319662D762D0130F70010
:100A900083165E08F8000319512D0310F70DF80BAB
:100AA0004D2D7708FF3A83128505762D0130F7002A
:100AB00083165E08F8000319612D0310F70DF80B7B
:100AC0005D2D7708FF3A83128605762D0130F700F9
:100AD00083165E08F8000319712D0310F70DF80B4B
:100AE0006D2D7708FF3A83128705762DC0308B0471
:100AF0000800861196308316DD0083123B22AD0A72
:100B00002919C42D2D080F3C0318C42DA91DB72D7C
:100B1000FF308500343083162A07840083130008D1
:100B2000A90083123A22A911033083169B002A08D8
:100B30009A009C131C1583120B08F7008B13831665
:100B400055309D00AA309D009C149C18A52D1C11A9
:100B5000770883128B0483162908DD008312670847
:100B60008316DE003C08DF008312A623C32D5F300E
:100B70008316E20083121B238316CD0183123C23CC
:100B80008316B5018312AD018A15F42983165A0B19
:100B9000CB2D0630DB00DA08031DD02D0230DB0040
:100BA000DC0158085C020318F22D0130DD005B08FF
:100BB000DE000130DF008312A62383165908DD0012
:100BC00083123B2201308316DD005B08DE00DF016B
:100BD0008312A62383165908DD0083123B22831655
:100BE000DC0AD12D8312080083165714400FF92D0B
:100BF000E32E6430DD0083123B2283164008063A60
:100C0000831203191C2E1B3A0319262E2B3A0319A3
:100C10002F2E213A0319392E073A0319472E013A8C
:100C20000319632E033A03197E2E013A03198A2E03
:100C3000073A0319962ECF2E0A308316D800323089
:100C4000D9000130DA008312C625CF2E0A30831670
:100C5000D8003230D900DA018312C625CF2E0130F8
:100C60008316D8003230D9000130DA008312C6254D
:100C7000CF2E01308316D8003230D900DA0183122A
:100C8000C6258316320B452EC2018312CF2E831642
:100C90002908153C031D552E831261088316D800C0
:100CA0001A30D9003930DA00612E0530D8003230E0
:100CB000D9000130DA008312C6258316320B612E6B
:100CC000B3018312CF2E83162908153C031D712E04
:100CD000831262088316D8001A30D9003930DA003E
:100CE000792E0530D8003230D900DA018312C625BA
:100CF0008316320B7C2EC2018312CF2E8316290855
:100D0000DD00831266088316DE003C08DF008312D4
:100D1000A623CF2E83162908DD00831267088316C9
:100D2000DE003C08DF008312A623CF2E8316B00816
:100D30000319B22EB001340BA92E290BA82E2908B5
:100D4000DD007108DE003C08DF008312A623831655
:100D5000B12E0130DD000330DE00DF018312A62357
:100D60008316CD2E0130B000340BC42E290BC32EB8
:100D70002908DD0083126E088316DE003C08DF00C0
:100D80008312A6238316CD2E0130DD000330DE0052
:100D90000130DF008312A62383168312CF2E831621
:100DA00056084002031DD82E4210FF30C000D92E35
:100DB0005710FF30C00083120A23003083165718E3
:100DC0000130F800E32E8312080001308316B200D0
:100DD000B60142146430DD0083123B2205308316D5
:100DE000D8003230D9000130DA008312C6250A2338
:100DF00083164D08CE00CF01B3014E08330203180D
:100E00001D2F0430D000FA30DD0083123B22831600
:100E1000D00B032FB30A8312291E122F2912831617
:100E2000FC2E831283164218172F1D2F1C2F4F08DC
:100E3000D6008312F4258316FD2E421C232F831225
:100E4000EE2E2A2F831683120A238316B2010C304A
:100E50008312AD00080083164008003A831203197C
:100E6000382F023A0319482F383A0319502F562FBA
:100E7000831629080A3C031D432F2830CD00831216
:100E8000E526472F83160630CD008312E526562F20
:100E900083162C08CD008A15831200288A11562F3C
:100EA00001308316CD0083125822562F8A15FC2953
:1010000003308316B20042143230DD008A1183129D
:101010003B228A1501308316B000340B1F28290BA0
:101020001E282908DD0083126E088316DE003C08A6
:10103000DF008A118312A6238A1583162A2801301D
:10104000DD000330DE000130DF008A118312A623A9
:101050008A158316CD08031DAB282C08CE00FE3060
:10106000CF008312A91283164E08D6007830D7001D
:10107000F701F801560803105718F707F70CF80C9A
:10108000D718F707F70CF80C5719F707F70CF80CF7
:10109000D719F707F70CF80C571AF707F70CF80CE5
:1010A000D71AF707F70CF80C571BF707F70CF80CD3
:1010B000D71BF707F70CF80C7808D2007708D30095
:1010C000D501D401D1010130D00051085302031CD5
:1010D000A828031D6F28520850020318A8280230C0
:1010E000D600FA30DD008A1183123B228A1583165E
:1010F000D60B71288312A91E7E28A928A91C8A282C
:10110000A910083083165007D4005108D5000318E1
:10111000D50A8312831654085002031D97285508D8
:101120005102031D9728831206168616831642184D
:101130009D288312A928A32883164F08D6008A1158
:101140008312F4258A158316D00A0319D10A65285B
:101150008312272983164D08CE00FE30CF0083125C
:10116000A91283164E08D6007830D700F701F8018F
:10117000560803105718F707F70CF80CD718F7079D
:10118000F70CF80C5719F707F70CF80CD719F707F5
:10119000F70CF80C571AF707F70CF80CD71AF707E3
:1011A000F70CF80C571BF707F70CF80CD71BF707D1
:1011B000F70CF80C7808D2007708D300D501D401D9
:1011C000D1010130D00051085302031C2629031D10
:1011D000ED2852085002031826290230D600FA30B2
:1011E000DD008A1183123B228A158316D60BEF2865
:1011F0008312A91EFC282729A91C0829A910083038
:1012000083165007D4005108D5000318D50A83125D
:10121000831654085002031D152955085102031D59
:101220001529831206168616831642181B29831267
:101230002729212983164F08D6008A118312F42505
:101240008A158316D00A0319D10AE328831283165C
:10125000B001340B3929290B38292908DD00710820
:10126000DE003C08DF008A118312A6238A1583164C
:1012700043290130DD000330DE00DF018A118312D3
:10128000A6238A158316B2018A1183120A238A15AE
:101290008A11562F840183131F30830583168E1500
:1012A00083128617BD01BE01BF012911A911A9171B
:1012B000CB1605308316C300F130C400E730C500FB
:1012C0002030C800D530C9008312CB1307309F00EF
:1012D0001F30B4000B30B5000730B6004630B70001
:1012E0000A30B8000C30B9000630BA001E30BB001E
:1012F0001430BC002910A9108A11A3298A15343092
:1013000083162A07840083130008A9008A11831218
:101310003A228A15AD0100306500FF3085000B13BD
:101320008B1283160108C0390238810007308312FE
:101330009F008316050885000330F700F70B9E29F0
:1013400083121F080C13FE306600061495309000BF
:101350008F0101308E000030650001306600831679
:10136000011383120B138B138B1BB3290613061166
:101370008611FF308500C6298A1150228A15013056
:101380008316CD008A11831258228A158B100B16F2
:101390008316011783128B108B100B16C0308B0431
:1013A0008A110A238A1503308316CA00CC01323011
:1013B000CB00FF30C0008312CB1DE4297608C300A8
:1013C000831623088312C40043088316B7008312D0
:1013D00029128A11192B8A158316CD018A118312BD
:1013E0003C238A158A11792D8A15291D1C2A8316FA
:1013F000B5018A1183122B2F8A158316400F032AF9
:10140000FF30C0001D2A4008D6008A118312F4253F
:101410008A158A110A238A157A308316E2008A1106
:1014200083121B238A157A308316E2008A118312F5
:101430001B238A15D0308B0483160230CD00FA307E
:10144000DD008A1183123B228A158316CD0B1F2AD9
:0E1450008A1183120A238A15F2292D2A6300BD
:0C42200001000200030004000400040080
:02400E00103F61
:00000001FF
